:100000000C942A000C940418189500001895000010
:100010000C94581C189500001895000018950000C5
:10002000189500001895000018950000189500001C
:10003000189500001895000018950000189500000C
:1000400018950000189500001895000018950000FC
:10005000189500008FE58DBFC0E4E0E14E2E84E0EE
:100060008EBFD4E0F4E05F2EEEEFF3E0A0E6B0E068
:10007000A89584B7082E877F84BF88E1992781BD22
:1000800091BD88278D933197E9F70E9493196624D3
:10009000DB9AE3E0F0E0A1E7B0E00E94711DE4E04C
:1000A000F0E0A4E7B0E00E94711D88EF8ABB8FE00A
:1000B00087BB83E084BB80EB81BB8FE482BB88E09D
:1000C00082BD85E085BD89B7806489BF83E886B934
:1000D00080EC87B98C9A83E38FBD81E08EBD8CE084
:1000E0000E94ED190E9478190E94041881E0809303
:1000F0008702009187020D3118F011F00C949E00D8
:10010000E7E8F2E0A190BB24E3E0F0E0AA0CBB1C1E
:10011000EA0DFB1DA7E8B2E0AD90BB24A3E7B0E079
:10012000AA0CBB1CAA0DBB1D0E94731DA7E8B2E060
:100130008C918F5F8C9310F40C94790081E0809304
:10014000870200918702033618F011F00C94CB005F
:10015000E7E8F2E0A190BB24EBE3F0E0AA0CBB1CC3
:10016000AA0CBB1CEA0DFB1DA7E8B2E0AD90BB24B6
:10017000AEEEB0E0AA0CBB1CAA0CBB1CAA0DBB1DAA
:1001800094E00E94741DA7E8B2E08C918F5F8C937D
:1001900010F40C94A100A0EDB0E0EEE5FBE30E94AA
:1001A000EE1BA1EEB0E0E0E7FBE30E94EE1BAFEA3E
:1001B000B0E0E2E8FBE30E94EE1BAAEBB0E0EEE861
:1001C000FBE30E94EE1BA5ECB0E0EAE9FBE30E9432
:1001D000EE1B0E94AA16C29A379A07B1007E0060F1
:1001E00007B90E94F41B082F192F003253E015079E
:1001F00010F00C9413018FE711E00E948719E6EAD2
:10020000FBE30E9471198FEB11E00E948719E8EB64
:10021000FBE30E947119E4E0F0E00E948A190C945B
:1002200082070C94430107B1007E006007B90E9469
:10023000F41B082F192F043853E0150710F00C9405
:1002400033018FE711E00E948719EAECFBE30E947B
:1002500071198FEB11E00E948719E8EBFBE30E9414
:1002600071190C9443018FE711E00E948719ECED9E
:10027000FBE30E9471198FEB11E00E948719EEEEEB
:10028000FBE30E9471193798C298E2E0F0E00E9407
:100290008A1980E08093880280E080939202A0E631
:1002A000B0E00E94261CC198C0988FE711E00E9420
:1002B0008719E0E0FCE30E9471198FEB11E00E94C6
:1002C0008719E2E1FCE30E9471190E94AA160E94BC
:1002D0009B168998AFE7B2E09C9194FF04C0819B84
:1002E00010C09F7E9C9381990CC084E69F939927B0
:1002F0000E94711A9F91819904C090619C930E9401
:100300003E0B8B98AFE7B2E09C9193FF04C0839BB8
:1003100010C0977F9C9383990CC084E69F93992784
:100320000E94711A9F91839904C098609C930E94C7
:100330005D0B00918802013011F00C94B9018A988C
:10034000AFE7B2E09C9192FF04C0829B10C09B7FFC
:100350009C9382990CC084E69F9399270E94711AFE
:100360009F91829904C094609C930C9476020C94A3
:100370006B02023011F00C94D7018A98AFE7B2E01B
:100380009C9192FF04C0829B10C09B7F9C9382999A
:100390000CC084E69F9399270E94711A9F918299BD
:1003A00004C094609C930C9477030C946B0203300C
:1003B00011F00C94F5018A98AFE7B2E09C9192FF9E
:1003C00004C0829B10C09B7F9C9382990CC084E6E2
:1003D0009F9399270E94711A9F91829904C09460FB
:1003E0009C930C94FE030C946B02043011F00C945B
:1003F00013028A98AFE7B2E09C9192FF04C0829BFF
:1004000010C09B7F9C9382990CC084E69F93992790
:100410000E94711A9F91829904C094609C930C94DD
:10042000EF050C946B02053011F00C9431028A98A0
:10043000AFE7B2E09C9192FF04C0829B10C09B7F0B
:100440009C9382990CC084E69F9399270E94711A0D
:100450009F91829904C094609C930C94D6070C944D
:100460006B02063011F00C944F028A98AFE7B2E0AD
:100470009C9192FF04C0829B10C09B7F9C938299A9
:100480000CC084E69F9399270E94711A9F918299CC
:1004900004C094609C930C9485040C946B02073008
:1004A00011F00C946B028A98AFE7B2E09C9192FF36
:1004B00004C0829B10C09B7F9C9382990CC084E6F1
:1004C0009F9399270E94711A9F91829904C094600A
:1004D0009C930C94FC04AFE7B2E08C9186FB16F081
:1004E0000C9474020C9486070C9469010E94E90B29
:1004F0000E949B168998AFE7B2E09C9194FF04C0DC
:10050000819B10C09F7E9C9381990CC084E69F9331
:1005100099270E94711A9F91819904C090619C93C0
:100520000E94E90B8B98AFE7B2E09C9193FF04C067
:10053000839B10C0977F9C9383990CC084E69F9304
:1005400099270E94711A9F91839904C098609C9387
:100550000E94080C8E98AFE7B2E09C9191FF04C016
:10056000869B10C09D7F9C9386990CC084E69F93C8
:1005700099270E94711A9F91869904C092609C935A
:100580000E94EF118898AFE7B2E09C9190FF04C001
:10059000809B10C09E7F9C9380990CC084E69F93A3
:1005A00099270E94711A9F91809904C091609C9331
:1005B0000E94ED0F00919202073011F00C94FA02A4
:1005C0008A98AFE7B2E09C9192FF04C0829B10C072
:1005D0009B7F9C9382990CC084E69F9399270E94ED
:1005E000711A9F91829904C094609C930C94C709DE
:1005F0000C946C03083011F00C9418038A98AFE740
:10060000B2E09C9192FF04C0829B10C09B7F9C93A0
:1006100082990CC084E69F9399270E94711A9F913A
:10062000829904C094609C930C94F5090C946C031B
:10063000093011F00C9436038A98AFE7B2E09C9130
:1006400092FF04C0829B10C09B7F9C9382990CC038
:1006500084E69F9399270E94711A9F91829904C002
:1006600094609C930C9441090C946C030A3011F033
:100670000C9454038A98AFE7B2E09C9192FF04C0B7
:10068000829B10C09B7F9C9382990CC084E69F93B1
:1006900099270E94711A9F91829904C094609C933B
:1006A0000C9482070C946C038A98AFE7B2E09C919B
:1006B00092FF04C0829B10C09B7F9C9382990CC0C8
:1006C00084E69F9399270E94711A9F91829904C092
:1006D00094609C930C944901AFE7B2E08C9186FB47
:1006E00016F00C9475030C9486070C947A020E9401
:1006F000240D0E949B168998AFE7B2E09C9194FF6D
:1007000004C0819B10C09F7E9C9381990CC084E69D
:100710009F9399270E94711A9F91819904C09061BB
:100720009C930E94240D8B98AFE7B2E09C9193FFBD
:1007300004C0839B10C0977F9C9383990CC084E670
:100740009F9399270E94711A9F91839904C0986082
:100750009C930E94430D8E98AFE7B2E09C9191FF6D
:1007600004C0869B10C09D7F9C9386990CC084E634
:100770009F9399270E94711A9F91869904C0926055
:100780009C930E94EF118898AFE7B2E09C9190FF94
:1007900004C0809B10C09E7F9C9380990CC084E60F
:1007A0009F9399270E94711A9F91809904C091602C
:1007B0009C930E94ED0F8A98AFE7B2E09C9192FF64
:1007C00004C0829B10C09B7F9C9382990CC084E6DE
:1007D0009F9399270E94711A9F91829904C09460F7
:1007E0009C930C944901AFE7B2E08C9186FB16F024
:1007F0000C94FC030C9486070C947B030E94750EEA
:100800000E949B168998AFE7B2E09C9194FF04C0C8
:10081000819B10C09F7E9C9381990CC084E69F931E
:1008200099270E94711A9F91819904C090619C93AD
:100830000E94750E8B98AFE7B2E09C9193FF04C0C5
:10084000839B10C0977F9C9383990CC084E69F93F1
:1008500099270E94711A9F91839904C098609C9374
:100860000E94940E8E98AFE7B2E09C9191FF04C075
:10087000869B10C09D7F9C9386990CC084E69F93B5
:1008800099270E94711A9F91869904C092609C9347
:100890000E94EF118898AFE7B2E09C9190FF04C0EE
:1008A000809B10C09E7F9C9380990CC084E69F9390
:1008B00099270E94711A9F91809904C091609C931E
:1008C0000E94ED0F8A98AFE7B2E09C9192FF04C0BE
:1008D000829B10C09B7F9C9382990CC084E69F935F
:1008E00099270E94711A9F91829904C094609C93E9
:1008F0000C944901AFE7B2E08C9186FB16F00C94A2
:1009000083040C9486070C9402040E94020E0E9439
:100910009B168998AFE7B2E09C9194FF04C0819B3D
:1009200010C09F7E9C9381990CC084E69F93992769
:100930000E94711A9F91819904C090619C930E94BA
:10094000020E8B98AFE7B2E09C9193FF04C0839BAB
:1009500010C0977F9C9383990CC084E69F9399273E
:100960000E94711A9F91839904C098609C930E9481
:10097000210E00919202033011F00C94D9048A9850
:10098000AFE7B2E09C9192FF04C0829B10C09B7FB6
:100990009C9382990CC084E69F9399270E94711AB8
:1009A0009F91829904C094609C930C9449010C948B
:1009B000F1048A98AFE7B2E09C9192FF04C0829B59
:1009C00010C09B7F9C9382990CC084E69F939927CB
:1009D0000E94711A9F91829904C094609C930E9416
:1009E000510AAFE7B2E08C9186FB16F00C94FA0442
:1009F0000C9486070C9489040E94500F0E949B1649
:100A00008998AFE7B2E09C9194FF04C0819B10C02D
:100A10009F7E9C9381990CC084E69F9399270E94A6
:100A2000711A9F91819904C090619C930E94500F0C
:100A30008B98AFE7B2E09C9193FF04C0839B10C0FA
:100A4000977F9C9383990CC084E69F9399270E947B
:100A5000711A9F91839904C098609C930E946F0FB4
:100A600000919202013011F00C9450058A98AFE782
:100A7000B2E09C9192FF04C0829B10C09B7F9C932C
:100A800082990CC084E69F9399270E94711A9F91C6
:100A9000829904C094609C930C9482070C94E405A2
:100AA000023011F00C946E058A98AFE7B2E09C9189
:100AB00092FF04C0829B10C09B7F9C9382990CC0C4
:100AC00084E69F9399270E94711A9F91829904C08E
:100AD00094609C930C94C7090C94E405033011F0C6
:100AE0000C948C058A98AFE7B2E09C9192FF04C009
:100AF000829B10C09B7F9C9382990CC084E69F933D
:100B000099270E94711A9F91829904C094609C93C6
:100B10000C94F5090C94E405043011F00C94AA052A
:100B20008A98AFE7B2E09C9192FF04C0829B10C00C
:100B30009B7F9C9382990CC084E69F9399270E9487
:100B4000711A9F91829904C094609C930C944109FE
:100B50000C94E405053011F00C94C8058A98AFE7B1
:100B6000B2E09C9192FF04C0829B10C09B7F9C933B
:100B700082990CC084E69F9399270E94711A9F91D5
:100B8000829904C094609C930C94270A0C94E40509
:100B9000063011F00C94E4058A98AFE7B2E09C911E
:100BA00092FF04C0829B10C09B7F9C9382990CC0D3
:100BB00084E69F9399270E94711A9F91829904C09D
:100BC00094609C930C944901AFE7B2E08C9186FB52
:100BD00016F00C94ED050C9486070C9400050E9409
:100BE0004A1780917F028F7780937F02A3E8B2E05B
:100BF0000E94261C85E080938702009187020D31B8
:100C000018F011F00C942206A3E8B2E00D911C91AB
:100C1000A7E8B2E0AD90BB24A3E7B0E0AA0CBB1CF0
:100C2000AA0DBB1D4D915C91040F151FA3E8B2E006
:100C30000D931C93A7E8B2E08C918D5F8C9310F418
:100C40000C94FD05A5E7B0E08D919C91A0E6B0E085
:100C50008D939C93A0E6B0E00D911C91003050E084
:100C6000150718F011F00C9437060C9469068FE7FD
:100C700011E00E948719A0EDB0E00E946B198FEB84
:100C800013E00E948719A8EFB3E0E0E6F0E00E94CD
:100C9000011D0E946919E4E2FCE30E9471198A981F
:100CA000AFE7B2E09C9192FF04C0829B10C09B7F93
:100CB0009C9382990CC084E69F9399270E94711A95
:100CC0009F91829904C094609C930C9449010C9468
:100CD0002A0681E08093890200918902093018F088
:100CE00011F00C946A07A9E8B2E00D91112743E0D6
:100CF00050E00E94C11BA5E8B2E00D931C93A5E84B
:100D0000B2E0AD90BC90A7E7B0E0AA0CBB1CAA0D66
:100D1000BB1D8D919C91A1E8B2E08D939C938FEBCC
:100D200011E00E948719E0E3FCE30E947119A1E839
:100D3000B2E00D911C91003050E0150718F011F051
:100D40000C94A4060C946207A5E8B2E0AD90BC90A8
:100D5000A3E7B0E0AA0CBB1CAA0DBB1D0D911C9112
:100D6000003050E0150718F011F00C94B9060C94FF
:100D7000580700917100013081E009F080E08F9305
:100D8000A7E7B0E00D911C91003050E0150780E01E
:100D900010F009F081E09F918923882311F40C94CD
:100DA000ED06A7E7B0E08D919C91A0E6B0E08D93B1
:100DB0009C930E94D8168FE711E00E948719A1EE3C
:100DC000B0E00E946B190E94E516009189020A307A
:100DD00011F00C94ED060C946A07A5E8B2E0AD9012
:100DE000BC90A3E7B0E0AA0CBB1CAA0DBB1D8D9163
:100DF0009C91A0E6B0E08D939C930E94D1168FE762
:100E000011E00E948719E2E4FCE30E947119A8EF47
:100E1000B3E0E9E8F2E00E94101D0E946919E8E4DD
:100E2000FCE30E9471190E94E516009189020A30C4
:100E300011F00C941D070C946A07A5E8B2E0AD9080
:100E4000BC90A5E7B0E0AA0CBB1CAA0DBB1D8D9100
:100E50009C91A0E6B0E08D939C93A0E6B0E00D914C
:100E60001C91003050E0150718F011F00C943A076F
:100E70000C9458078FE711E00E948719E2E4FCE325
:100E80000E947119A8EFB3E0E9E8F2E00E94101D9A
:100E90000E946919E4E5FCE30E9471190E94E516BD
:100EA000009189020A3011F00C9458070C946A07DB
:100EB000A1E8B2E00E940919A3E8B2E00E94091972
:100EC0000C949706A9E8B2E08C918F5F8C9310F494
:100ED0000C946C068FE711E00E948719E0E6FCE3B2
:100EE0000E9471198FEB11E00E948719E2E7FCE381
:100EF0000E9471190E94AA16E4E0F0E00E948A198B
:100F00000C94E9000E944A17DB98D3980E94781944
:100F10008FE711E00E948719E4E8FCE30E94711951
:100F20008FEB15E00E9487190E94801AA2EAB2E0B6
:100F30000E946B198C988BB780648BBF85B78C7FB0
:100F400085BF80917F02806480937F0287E0E4EF19
:100F5000F1E0A2E30E94381C85B7806785BF8895C1
:100F6000AFE7B2E08C9186FB0EF4F0CFE3E9F2E05C
:100F70000E94431BA0E1B0E00D911D912D913C9189
:100F800041E050E060E070E00E94E41CACE8B2E0B8
:100F90000D931D932D933D93ECE8F2E0A2EAB2E0AD
:100FA0000E94B91B0E94891A0C94E9000E944A17FA
:100FB00080917F028F7780937F0281E080939202FD
:100FC00081E08093960281E08093970280E0809395
:100FD00098024FEF5FEF6FEF7FEFA2E9B2E0AD90C5
:100FE000BB24AEEEB0E0AA0CBB1CAA0CBB1CAA0D25
:100FF000BB1D0D911D912D913C910E94EE1C80E036
:1010000014F009F081E08F9300919202043681E0A0
:1010100008F080E09F918923882311F40C9429091A
:1010200000917100013081E009F080E08F93A7E723
:10103000B0E00D911C91003050E0150780E010F0F9
:1010400009F081E09F918923882311F40C944808CA
:10105000A2E9B2E0AD90BB24AEEEB0E0AA0CBB1C9E
:10106000AA0CBB1CAA0DBB1D0D911D912D913C918D
:10107000A7E7B0E04D915C91662777270E94E91CB5
:10108000ACE8B2E00D931D932D933D930C945E0854
:10109000A2E9B2E0AD90BB24AEEEB0E0AA0CBB1C5E
:1010A000AA0CBB1CAA0DBB1D0D911D912D913C914D
:1010B000ACE8B2E00D931D932D933C938FEB11E0C0
:1010C0000E948719E6E9FCE30E947119E2E9F2E067
:1010D000A190BB24EEEEF0E0AA0CBB1CAA0CBB1C3A
:1010E000EA0DFB1DA8EFB3E00E94B91B0E9469192D
:1010F0008FE711E00E948719EEE9FCE30E94711965
:101100000E94801AA2EAB2E00E946B198A98AFE7A7
:10111000B2E09C9192FF04C0829B10C09B7F9C9385
:1011200082990CC084E69F9399270E94711A9F911F
:10113000829904C094609C930C94E900E3E9F2E086
:101140000E94801BA0E1B0E04D915D916D917C917A
:10115000ACE8B2E00D911D912D913C910E94EE1CE6
:1011600011F00C94780800917100013081E009F0D1
:1011700080E08F93A7E7B0E00D911C91003050E024
:10118000150780E010F009F081E09F918923882302
:1011900011F40C9412090E94D8168FE711E00E94F6
:1011A0008719E6EAFCE30E9471190E94801AA2EAFC
:1011B000B2E00E946B198A98AFE7B2E09C9192FF6F
:1011C00004C0829B10C09B7F9C9382990CC084E6D4
:1011D0009F9399270E94711A9F91829904C09460ED
:1011E0009C930C94E900E3E9F2E00E94801BA0E1EB
:1011F000B0E04D915D916D917C91A2E9B2E0AD902E
:10120000BB24AEEEB0E0AA0CBB1CAA0CBB1CAA0D02
:10121000BB1D0D911D912D913C910E94EE1C11F072
:101220000C94CD088FE711E00E948719EEEAFCE3E9
:101230000E9471190E94801AA2EAB2E00E946B1902
:101240000E94D816A2E9B2E08C918F5F8C930C9427
:10125000E9078FE711E00E948719E6EBFCE30E94A3
:1012600071198FEB11E00E948719E2E7FCE30E94FD
:1012700071190E94AA16E4E0F0E00E948A190C9409
:10128000E9008FEB11E00E948719E8ECFCE30E9473
:1012900071190E94AA1681E080938702009187024B
:1012A0000D3118F011F00C947409E7E8F2E0A19008
:1012B000BB24E3E0F0E0AA0CBB1CEA0DFB1DA7E891
:1012C000B2E0AD90BB24A3E7B0E0AA0CBB1CAA0D12
:1012D000BB1D7BE70E94621DA7E8B2E08C918F5F87
:1012E0008C9310F40C944E0981E080938702009156
:1012F0008702033618F011F00C94A209E7E8F2E037
:10130000A190BB24EBE3F0E0AA0CBB1CAA0CBB1C15
:10131000EA0DFB1DA7E8B2E0AD90BB24AEEEB0E055
:10132000AA0CBB1CAA0CBB1CAA0DBB1D94E07BE73E
:101330000E94631DA7E8B2E08C918F5F8C9310F43C
:101340000C947709E0E0F0E0AEE6B0E07BE70E94C5
:10135000601DE1E0F0E0AFE6B0E07BE70E94601DD9
:10136000E2E0F0E0A0E7B0E07BE70E94601DE3E090
:10137000F0E0A1E7B0E07BE70E94601DE4E0F0E070
:10138000A4E7B0E07BE70E94601D0C9449018FEB5D
:1013900011E00E948719EAEDFCE30E9471190E9496
:1013A000AA1681E080938702009187020D3118F020
:1013B00011F00C94EF09A7E8B2E0AD90BB24A3E7CD
:1013C000B0E0AA0CBB1CAA0DBB1D0E94261CA7E8FE
:1013D000B2E08C918F5F8C9310F40C94D409E2E00E
:1013E000F0E00E948A190C9449018FEB11E00E94F1
:1013F0008719ECEEFCE30E9471190E94AA1681E0A5
:101400008093870200918702033618F011F00C9444
:10141000210AA7E8B2E0AD90BB24AEEEB0E0AA0C82
:10142000BB1CAA0CBB1CAA0DBB1DE6E1FBE30E9482
:10143000161CA7E8B2E08C918F5F8C9310F40C948B
:10144000020AE2E0F0E00E948A190C9449018FE759
:1014500011E00E948719EEEFFCE30E9471198FEBF7
:1014600011E00E948719E0E1FDE30E9471190E94DA
:101470009B160E9485168FE711E00E948719E2E211
:10148000FDE30E9471198FEB11E00E948719E4E3DC
:10149000FDE30E9471190E949B160E9485160C9410
:1014A00049018FE711E00E948719E6E4FDE30E94FD
:1014B00071198FEB11E00E948719E8E5FDE30E94A6
:1014C00071190E94AA160E949B160E948516C19A45
:1014D00000917100013011F00C947E0A8FE711E049
:1014E0000E948719E0E7FBE30E9471190E94AA1687
:1014F0000E949B160E9485160E94D81600919202A7
:10150000013011F00C94D90A8FE711E00E9487197D
:10151000EAE6FDE30E9471190E94AA160E949B163A
:101520000E9485160E944A178FE711E00E948719D2
:10153000ECE7FDE30E9471198FEB11E00E9487191F
:10154000E6E8FDE30E9471190E94AA1680917F02CD
:101550008F7780937F02A0E6B0E00E94261C0E9455
:10156000D116A0E3B0E00C9102FB0EF016C08FE79D
:101570001BE00E948719A8EFB3E0E0E6F0E00E94CC
:10158000011D0E946919E8E9FDE30E94711984E6D2
:1015900090E00E94711A0C94B10A8FE711E00E944A
:1015A0008719EAE9FDE30E9471190E94AA160C94BA
:1015B0002F0B023011F00C942F0B8FE711E00E94DB
:1015C0008719ECEAFDE30E9471198FEB11E00E948C
:1015D0008719EEEBFDE30E9471190E94AA160E9482
:1015E0009B160E9485160E9478198FE711E00E94D1
:1015F0008719E0EDFDE30E9471190E94AA16A0E68A
:10160000B0E00E94261C0E94D116A0E3B0E00C912D
:1016100002FB0EF41CC08FEB11E00E948719E2EE72
:10162000FDE30E947119A8EFB3E0E0E6F0E00E944C
:10163000011D0E946919E8E9FDE30E9471190E94E9
:10164000AA1684E690E00E94711A0C94050B8FE7AD
:1016500011E00E948719EEEEFDE30E947119C09817
:10166000C1988FEB11E00E948719E0E0FEE30E9431
:1016700071190E94AA160E949B160895A8E8B2E06C
:101680008C918F5F8C9300918802073080E010F07E
:1016900009F081E08F9300918802013081E008F029
:1016A00080E09F91892B882311F40C945A0B81E0E0
:1016B000809388020E947C0B08958091880281505B
:1016C0008093880200918802013081E008F080E078
:1016D0008F9300918802073080E010F009F081E0DC
:1016E0009F91892B882311F40C94790B87E08093C8
:1016F00088020E947C0B089500918802013011F04D
:101700000C948C0B8FE711E00E948719E2E1FEE355
:101710000E9471190C94DE0B023011F00C949A0B9C
:101720008FE711E00E948719E4E2FEE30E9471193D
:101730000C94DE0B033011F00C94A80B8FE711E032
:101740000E948719E6E3FEE30E9471190C94DE0BF8
:10175000043011F00C94B60B8FE711E00E9487194A
:10176000E0E6FCE30E9471190C94DE0B053011F0E9
:101770000C94C40B8FE711E00E948719E6EBFCE3A1
:101780000E9471190C94DE0B063011F00C94D20BF0
:101790008FE711E00E948719ECEAFDE30E947119BE
:1017A0000C94DE0B073011F00C94DE0B8FE711E088
:1017B0000E948719E8E4FEE30E9471198FEB11E0A3
:1017C0000E948719E0E0FEE30E9471190E94AA16A8
:1017D0000895A2E9B2E08C918F5F8C930091920200
:1017E000063080E010F009F081E08F9300919202C2
:1017F000013081E008F080E09F91892B882311F46B
:101800000C94050C81E0809392020E94270C0895AD
:101810008091920281508093920200919202013055
:1018200081E008F080E08F9300919202063080E022
:1018300010F009F081E09F91892B882311F40C941A
:10184000240C86E0809392020E94270C08950E9447
:10185000781900919202013011F00C94470C8FE737
:1018600011E00E948719EAE5FEE30E9471198FEBEF
:1018700018E00E948719A8EFB3E0E0E7F0E00E94CB
:10188000101D0E9469190E94AA160C94230D0230A3
:1018900011F00C947E0C8FEF80937E028FE711E0A5
:1018A0000E948719ECE6FEE30E9471198FEB18E0A5
:1018B0000E948719A8EFB3E0EEE6F0E00E94101D49
:1018C0000E94691902E010E0AEE6B0E04D915527A4
:1018D0000E945019AAE8B2E00D931C93AAE8B2E066
:1018E0000D911C9141E050E0041B150BA0E1B0E00C
:1018F0008D919C9199BD88BD0C94230D033011F0FE
:101900000C94B50C8FEF80937E028FE711E00E945C
:101910008719EEE7FEE30E9471198FEB18E00E9431
:101920008719A8EFB3E0EFE6F0E00E94101D0E94D7
:10193000691902E010E0AFE6B0E04D9155270E9432
:101940005019AAE8B2E00D931C93AAE8B2E00D91F9
:101950001C9141E050E0041B150BA0E1B0E08D911B
:101960009C9199BD88BD0C94230D043011F00C940A
:10197000D90C80917F02806280937F028FE711E013
:101980000E948719E0E9FEE30E9471198FEB15E0D0
:101990000E9487190E94801AA2EAB2E00E946B1985
:1019A00080917F028F7D80937F020E94AA160C9403
:1019B000230D053011F00C94050D8FE711E00E9406
:1019C0008719E2EAFEE30E9471190091710000306C
:1019D00011F00C94F50C8FEB11E00E948719E4EBE9
:1019E000FEE30E9471190C94010D013011F00C946A
:1019F000010D8FEB11E00E948719E6ECFEE30E94D7
:101A000071190E94AA160C94230D063011F00C9443
:101A1000230D8FE711E00E948719E8EDFEE30E9495
:101A200071198FEB14E00E948719A8EFB3E0E4E787
:101A3000F0E00E94101D0E946919EAEEFEE30E9488
:101A400071190E94AA160895A2E9B2E08C918F5FE5
:101A50008C93009192020D3180E010F009F081E04A
:101A60008F9300919202013081E008F080E09F9115
:101A7000892B882311F40C94400D81E0809392020D
:101A80000E94620D0895809192028150809392028B
:101A900000919202013081E008F080E08F93009184
:101AA00092020D3180E010F009F081E09F91892BC6
:101AB000882311F40C945F0D8DE1809392020E94B3
:101AC000620D08950E94781900919202033010F07F
:101AD0000C947E0D8FE711E00E948719A2E9B2E015
:101AE0000D91112741E150E00E94C11BAFEBB0E026
:101AF000A00FB11F0E946B190C94B50D00919202BA
:101B000043E00E947B1DA9E8B2E00C938FE711E04F
:101B10000E948719E2E4FCE30E947119A8EFB3E088
:101B2000E9E8F2E00E94101D0E94691900919202FA
:101B300043E00E947B1DA9E8B2E08C93A9E8B2E0E3
:101B40008C918F5F8C938FE717E00E948719A9E82B
:101B5000B2E00D9111274BE050E00E94C11BA4EAB6
:101B6000B0E0A00FB11F0E946B190091920243E0F8
:101B70000E947B1DA9E8B2E08C930091890202309B
:101B800081E009F080E08F9300919202023080E0C2
:101B900010F009F081E09F918923882311F40C94BF
:101BA000E70D8FEB18E00E948719A8EFB3E0E2E998
:101BB000F2E0A190BB24E3E7F0E0AA0CBB1CEA0D25
:101BC000FB1D0E94011D0E9469190C94FF0D8FEBF3
:101BD00013E00E948719A8EFB3E0E2E9F2E0A190D8
:101BE000BB24E3E7F0E0AA0CBB1CEA0DFB1D0E943E
:101BF000011D0E946919E4EFFEE30E9471190E9421
:101C0000AA160895A2E9B2E08C918F5F8C9300919F
:101C10009202033080E010F009F081E08F93009190
:101C20009202013081E008F080E09F91892B8823A7
:101C300011F40C941E0E81E0809392020E94400EDB
:101C400008958091920281508093920200919202B5
:101C5000013081E008F080E08F9300919202033020
:101C600080E010F009F081E09F91892B882311F426
:101C70000C943D0E83E0809392020E94400E0895E2
:101C800000919202013011F00C94500E8FE711E098
:101C90000E948719EAE9FDE30E9471190C946A0E0B
:101CA000023011F00C945E0E8FE711E00E9487194C
:101CB000EEEEFDE30E9471190C946A0E033011F0F0
:101CC0000C946A0E8FE711E00E948719EEEFFEE395
:101CD0000E9471198FEB11E00E948719E0E0FEE38A
:101CE0000E9471190E94AA160895A2E9B2E08C918F
:101CF0008F5F8C9300919202033680E010F009F020
:101D000081E08F9300919202013081E008F080E041
:101D10009F91892B882311F40C94910E81E080937C
:101D200092020E94B30E0895809192028150809396
:101D3000920200919202013081E008F080E08F93DE
:101D400000919202033680E010F009F081E09F914B
:101D5000892B882311F40C94B00E83E680939202B1
:101D60000E94B30E08950E9478198FE711E00E9437
:101D70008719E0E1FFE30E947119A8EFB3E0E2E9FF
:101D8000F2E00E94101D0E94691940E050E060E0FE
:101D900070E0A2E9B2E0AD90BB24AEEEB0E0AA0CD8
:101DA000BB1CAA0CBB1CAA0DBB1D0D911D912D9136
:101DB0003C910E94EE1C0CF402C00C94E90E8FEBD7
:101DC00011E00E948719EEE1FFE30E9471190C9463
:101DD0004D0F40E851E561E070E0A2E9B2E0AD905E
:101DE000BB24AEEEB0E0AA0CBB1CAA0CBB1CAA0D17
:101DF000BB1D0D911D912D913C910E94EE1C0CF488
:101E000002C00C941B0F8FEB15E00E948719E2E9CA
:101E1000F2E0A190BB24EEEEF0E0AA0CBB1CAA0CF1
:101E2000BB1CEA0DFB1DA8EFB3E00E94B91B0E948A
:101E300069190C944D0F8FEB13E00E948719E2E9AA
:101E4000F2E0A190BB24EEEEF0E0AA0CBB1CAA0CC1
:101E5000BB1CEA0DFB1DA8EFB3E00E94B91B0E945A
:101E60006919E0E3FFE30E947119E2E9F2E0A19051
:101E7000BB24EEEEF0E0AA0CBB1CAA0CBB1CEA0DC6
:101E8000FB1D0E943F1B002F112FA8EFB3E0E0E1E4
:101E9000F0E00E94011D0E9469190E94AA1608958F
:101EA000A2E9B2E08C918F5F8C9300919202063090
:101EB00080E010F009F081E08F93009192020130F0
:101EC00081E008F080E09F91892B882311F40C9425
:101ED0006C0F81E0809392020E948E0F0895809192
:101EE000920281508093920200919202013081E02F
:101EF00008F080E08F9300919202063080E010F0AD
:101F000009F081E09F91892B882311F40C948B0FA9
:101F100086E0809392020E948E0F089500919202B3
:101F2000013011F00C949E0F8FE711E00E94871989
:101F3000E4E3FFE30E9471190C94E20F023011F008
:101F40000C94AC0F8FE711E00E948719E6E4FFE3E1
:101F50000E9471190C94E20F033011F00C94BA0F27
:101F60008FE711E00E948719E8E5FFE30E947119ED
:101F70000C94E20F043011F00C94C80F8FE711E0BD
:101F80000E948719EAE6FFE30E9471190C94E20FA0
:101F9000053011F00C94D60F8FE711E00E948719DD
:101FA000ECE7FFE30E9471190C94E20F063011F088
:101FB0000C94E20F8FE711E00E948719EEEFFEE329
:101FC0000E9471198FEB11E00E948719E0E0FEE397
:101FD0000E9471190E94AA16089580E080938002E1
:101FE00000918802013011F00C9488100091920247
:101FF000013011F00C940E10A0E7B0E08C91A2E635
:10200000B0E08D9388278D938D938C93AAE6B0E0F2
:10201000EAE1FBE30E94161C0C948610023011F0DA
:102020000C942810AEE6B0E08C91A2E6B0E08D935F
:1020300088278D938D938C93AFE6B0E08C91AAE6C0
:10204000B0E08D9388278D938D938C930C9486109C
:10205000033011F00C943E10AFE6B0E08C91A2E694
:10206000B0E08D9388278D938D938C93AAE6B0E092
:10207000EEE1FBE30E94161C0C948610043011F074
:102080000C945C10E3E9F2E00E94431BA2E6B0E08E
:102090000D931D932D933D9380E080938702809153
:1020A0007F02806280937F02AAE6B0E0E2E2FBE377
:1020B0000E94161C0C948610053011F00C947210BE
:1020C000A1E7B0E08C91A2E6B0E08D9388278D93D4
:1020D0008D938C93AAE6B0E0E6E2FBE30E94161C27
:1020E0000C948610063011F00C948610A4E7B0E032
:1020F0008C91A2E6B0E08D9388278D938D938C937D
:10210000AAE6B0E0EAE2FBE30E94161C0C9465111B
:10211000023011F00C94B510A2E9B2E0AD90BB24EE
:10212000A3E7B0E0AA0CBB1CAA0DBB1D8D919C912E
:10213000A2E6B0E08D939D9388278D938C930091B8
:102140009202023011F00C94AD10AAE6B0E0EEE27B
:10215000FBE30E94161C0C94B310AAE6B0E0E2E385
:10216000FBE30E94161C0C946511033011F00C94D3
:102170006511A2E9B2E0AD90BB24AEEEB0E0AA0CCE
:10218000BB1CAA0CBB1CAA0DBB1D0D911D912D9152
:102190003C91A2E6B0E00D931D932D933C930091EA
:1021A0009202013011F00C94E110E3E9F2E00E9498
:1021B000431BA6E6B0E00D931D932D933D930C9425
:1021C000FD10A2E9B2E0AD90BB24AAEEB0E0AA0CEB
:1021D000BB1CAA0CBB1CAA0DBB1D0D911D912D9102
:1021E0003C9149E050E060E070E00E94E41CA6E60B
:1021F000B0E00D931D932D933D93A6E6B0E04D9175
:102200005D916D917C91A2E6B0E00D911D912D91B3
:102210003C910E94EE1C0CF402C00C941B11A6E62B
:10222000B0E00D911D912D913C91A2E6B0E00D938F
:102230001D932D933C9300919202033681E009F0A7
:1022400080E08F934FEF5FEF6FEF7FEFA2E9B2E097
:10225000AD90BB24A2EFB0E0AA0CBB1CAA0CBB1C27
:10226000AA0DBB1D0D911D912D913C910E94EE1C5C
:1022700081E009F080E09F91892B882311F40C9470
:102280004911AAE6B0E0E6E3FBE30E94161C0C94B9
:102290006511A2E9B2E0AD90BB24A2EFB0E0AA0CB8
:1022A000BB1CAA0CBB1CAA0DBB1D0D911D912D9131
:1022B0003C914AE050E060E070E00E94E91CAAE630
:1022C000B0E00D931D932D933D93A0E3B0E00C91EE
:1022D00000FB81E00EF480E08F93AAE6B0E04D9120
:1022E0005D916D917C91A2E6B0E00D911D912D91D3
:1022F0003C910E94EE1C80E00CF481E09F918923C8
:10230000882311F40C94E9110E947117A2E6B0E041
:102310000D911D912D913C91ACE8B2E04D915D91F4
:102320006D917C910E94E41CA2E6B0E00D931D9398
:102330002D933D93AAE6B0E04D915D916D917C9116
:10234000A2E6B0E00D911D912D913C910E94EE1CF2
:102350001CF011F00C94AE110C94BA11AAE6B0E086
:102360000D911D912D913C91A2E6B0E00D931D932E
:102370002D933C9300918802013081E009F080E0C8
:102380008F9300919202043081E009F080E09F91E8
:1023900089238F93AAE6B0E04D915D916D917C9178
:1023A000A2E6B0E00D911D912D913C910E94EE1C92
:1023B00081E009F080E09F918923882311F40C9437
:1023C000E511A2E6B0E00E94281C0E94D2130C94F2
:1023D000651180917F028F7D80937F02089580E058
:1023E0008093800200918802013011F00C948412D5
:1023F00000919202013011F00C940E12A0E7B0E0AF
:102400008C91A2E6B0E08D9388278D938D938C9369
:10241000A6E6B0E00E94281C0C948212023011F053
:102420000C942212AEE6B0E08C91A2E6B0E08D935F
:1024300088278D938D938C93A6E6B0E00E94281C8C
:102440000C948212033011F00C943C12AFE6B0E011
:102450008C91A2E6B0E08D9388278D938D938C9319
:10246000AEE6B0E08C91A6E6B0E08D9388278D9320
:102470008D938C930C948212043011F00C945A12A8
:10248000E3E9F2E00E94431BA2E6B0E00D931D9346
:102490002D933D9380E08093870280917F0280623C
:1024A00080937F02A6E6B0E0E6E1FBE30E94161C03
:1024B0000C948212053011F00C946E12A1E7B0E07A
:1024C0008C91A2E6B0E08D9388278D938D938C93A9
:1024D000A6E6B0E00E94281C0C948212063011F08F
:1024E0000C948212A4E7B0E08C91A2E6B0E08D9348
:1024F00088278D938D938C93A6E6B0E0E6E2FBE30C
:102500000E94161C0C942713023011F00C94A11297
:10251000A2E9B2E0AD90BB24A3E7B0E0AA0CBB1CDB
:10252000AA0DBB1D8D919C91A2E6B0E08D939D9369
:1025300088278D938C93A6E6B0E00E94281C0C940B
:102540002713033011F00C942713A2E9B2E0AD90E9
:10255000BB24AEEEB0E0AA0CBB1CAA0CBB1CAA0D9F
:10256000BB1D0D911D912D913C91A2E6B0E00D9304
:102570001D932D933C9300919202013081E009F06C
:1025800080E08F934FEF5FEF6FEF7FEFA2E9B2E054
:10259000AD90BB24AAEEB0E0AA0CBB1CAA0CBB1CDD
:1025A000AA0DBB1D0D911D912D913C910E94EE1C19
:1025B00081E009F080E09F91892B882311F40C942D
:1025C000ED12E3E9F2E00E94431BA6E6B0E00D93B2
:1025D0001D932D933D930C942713A2E9B2E0AD9087
:1025E000BB24AAEEB0E0AA0CBB1CAA0CBB1CAA0D13
:1025F000BB1D0D911D912D913C9149E050E060E093
:1026000070E00E94E41CA6E6B0E00D931D932D93AC
:102610003D93A6E6B0E04D915D916D917C91A2E66F
:10262000B0E00D911D912D913C910E94EE1C0CF497
:1026300002C00C942713A6E6B0E00D911D912D91D8
:102640003C91A2E6B0E00D931D932D933C93A0E343
:10265000B0E00C9106FB81E00EF480E08F93A6E6DB
:10266000B0E04D915D916D917C91A2E6B0E00D914D
:102670001D912D913C910E94EE1C80E014F009F018
:1026800081E09F918923882311F40C94CC130E943C
:102690007117A2E6B0E00D911D912D913C91ACE82F
:1026A000B2E04D915D916D917C910E94E91CA2E692
:1026B000B0E00D931D932D933D930091880203305C
:1026C00011F00C947D13A6E6B0E04D915D916D91F3
:1026D0007C91A2E6B0E00D911D912D913C910E945C
:1026E000EE1C1CF011F00C947B13A2E6B0E0E6E1C6
:1026F000FBE30E94161C0C949B13A6E6B0E04D91E0
:102700005D916D917C91A2E6B0E00D911D912D91AE
:102710003C910E94EE1C0CF402C00C949B13A6E6A4
:10272000B0E00D911D912D913C91A2E6B0E00D938A
:102730001D932D933C9300918802013081E009F0B4
:1027400080E08F9300919202043081E009F080E0F4
:102750009F9189238F93A6E6B0E04D915D916D9195
:102760007C91A2E6B0E00D911D912D913C910E94CB
:10277000EE1C81E009F080E09F918923882311F409
:102780000C94C813A2E6B0E0EAE3FBE30E94161C37
:102790000E94D2130C94271380917F028F7D809327
:1027A0007F0208958FEB11E00E948719E0E3FCE3BC
:1027B0000E94711900918802013011F00C94E51407
:1027C00000919202013011F00C94FC138091620090
:1027D000809370000E94A8188FEB18E00E94871960
:1027E000A8EFB3E0E2E6F0E00E94041D0E94691940
:1027F0000E94AA160C94E314023011F00C942F14CA
:102800008FEF80937E028091620080936E0002E0E1
:1028100010E0AEE6B0E04D9155270E945019AAE8AD
:10282000B2E00D931C93AAE8B2E00D911C9141E037
:1028300050E0041B150BA0E1B0E08D919C9199BD77
:1028400088BD8FEB18E00E948719A8EFB3E0E2E69D
:10285000F0E00E94041D0E9469190C94E3140330F7
:1028600011F00C9462148FEF80937E0280916200CD
:1028700080936F0002E010E0AFE6B0E04D91552785
:102880000E945019AAE8B2E00D931C93AAE8B2E0A6
:102890000D911C9141E050E0041B150BA0E1B0E04C
:1028A0008D919C9199BD88BD8FEB18E00E9487198E
:1028B000A8EFB3E0E2E6F0E00E94041D0E9469196F
:1028C0000C94E314043011F00C949314A2E6B0E0DD
:1028D0000D911D912D913C91A7E8B2E04C915527A7
:1028E000662777270E94E41CA2E6B0E00D931D93B3
:1028F0002D933D9380E080938702E2E6F0E0A2EA28
:10290000B2E00E94B91B0E94891A8FEB15E00E9469
:1029100087190E94801AA2EAB2E00E946B190E94F5
:10292000AA160C94E314053011F00C94C91480918C
:1029300062008093710040E050E060E070E0A2E649
:10294000B0E00D911D912D913C910E94EE1C11F073
:102950000C94B4148FEB11E00E948719E4EBFEE3B2
:102960000E9471190C94C51441E050E060E070E0E1
:102970000E94EE1C11F00C94C5148FEB11E00E9424
:102980008719E6ECFEE30E9471190E94AA160C94C6
:10299000E314063011F00C94E314809162008093EC
:1029A00074008FEB14E00E948719A8EFB3E0E2E611
:1029B000F0E00E94041D0E946919EAEEFEE30E9405
:1029C00071190E94AA160C94A915023011F00C94EA
:1029D0003715A2E6B0E08D919C91A2E9B2E0AD90EE
:1029E000BB24A3E7B0E0AA0CBB1CAA0DBB1D8D93B2
:1029F0009C930091920243E00E947B1DA9E8B2E003
:102A00008C9300918902023081E009F080E08F937D
:102A100000919202023080E010F009F081E09F9175
:102A20008923882311F40C9423158FEB18E00E945E
:102A30008719A8EFB3E0E2E6F0E00E94041D0E94CF
:102A400069190C9433158FEB13E00E948719A8EFD6
:102A5000B3E0E2E6F0E00E94041D0E946919E4EF91
:102A6000FEE30E9471190E94AA160C94A915033066
:102A700011F00C94A915A2E6B0E00D911D912D91D5
:102A80003C91A2E9B2E0AD90BB24AEEEB0E0AA0C5E
:102A9000BB1CAA0CBB1CAA0DBB1D0D931D932D9333
:102AA0003C9340E050E060E070E0A2E6B0E00D91C1
:102AB0001D912D913C910E94EE1C0CF402C00C94CF
:102AC0006B158FEB11E00E948719EEE1FFE30E9486
:102AD00071190C94A71540E851E561E070E0A2E699
:102AE000B0E00D911D912D913C910E94EE1C0CF4D3
:102AF00002C00C9489158FEB15E00E948719E2E65D
:102B0000F0E0A8EFB3E00E94B91B0E9469190C9491
:102B1000A7158FEB13E00E948719E2E6F0E0A8EF1B
:102B2000B3E00E94B91B0E946919E0E3FFE30E9431
:102B30007119E2E6F0E00E943F1B002F112FA8EF71
:102B4000B3E0E0E1F0E00E94011D0E9469190E94DB
:102B5000AA1684E690E00E94711A0895AFE7B2E0E9
:102B60008C9186FB16F00C94C1158FEB15E00E943A
:102B700087190E94801AA2EAB2E00E946B190C9495
:102B8000841600917E020F3F11F00C94CA150000CC
:102B90000C940B1600917E02053010F00C94F11588
:102BA000AEE7B2E08C918F5F8C9302E010E0AFE66D
:102BB000B0E04D9155270E945019A0E9B2E00D9365
:102BC0001C93A0E9B2E00D911C9141E050E0041B80
:102BD000150BA0E1B0E08D919C9199BD88BD0C943E
:102BE0000B1602E010E0AEE6B0E04D9155270E94D2
:102BF0005019A0E9B2E00D931C93A0E9B2E00D9149
:102C00001C9141E050E0041B150BA0E1B0E08D9158
:102C10009C9199BD88BDAFE7B2E08C9187FB16F01F
:102C20000C943616A2E7B0E00D911C914CE350E0F5
:102C30000E943619A0E9B2E04D935C93A4E7B0E09E
:102C40004D915527A0E9B2E00D911C91041715078D
:102C500010F40C94321680917F02806480937F027E
:102C60000C943616A2E7B0E00E940219009180028F
:102C7000023310F00C944116A0E8B2E08C918F5F03
:102C80008C9300918802013011F00C94651600912C
:102C90009202043011F00C946316A7E8B2E08C9114
:102CA0008F5F8C93AFE7B2E08C9185FB16F40C94A8
:102CB00063168FEB15E00E9487190E94801AA2EA22
:102CC000B2E00E946B190C948416043011F00C943D
:102CD0007C16A0E6B0E00D911C91003050E0150785
:102CE00018F011F00C9476160C947A16A0E6B0E069
:102CF0000E9409190C948416063011F00C94841665
:102D0000A0E6B0E00E9402190895A0E3B0E00C91A3
:102D100002FB0EF00FC0AFE7B2E08C9186FB16F01D
:102D20000C9494160C94860784E690E00E94711A25
:102D30000C9485160895A0E3B0E00C9102FB0EF40C
:102D400008C00E94AA1684E690E00E94711A0C94B2
:102D50009B160895A2E7B0E00E94261C80917F0296
:102D6000806880937F0280E080937E0202E010E022
:102D7000AFE6B0E04D9155270E945019AAE8B2E0A5
:102D80000D931C93AAE8B2E00D911C9141E050E034
:102D9000041B150BA0E1B0E08D919C9199BD88BDFD
:102DA0000895C19A88EC90E00E94711AC09A089523
:102DB000C19A88EC90E00E94711A80E0E8EFF4E29A
:102DC000A8E30E94381CC1980895A0E6B0E00D91D8
:102DD0001C91003050E0150718F011F00C94F21619
:102DE0000C943F178FEB11E00E948719A8EFB3E016
:102DF000E0E6F0E00E94011D0E946919EEE8FFE3A1
:102E00000E9471198FEB17E00E948719A8EFB3E0B9
:102E1000E1E8F2E00E94011D0E946919E2E9FFE386
:102E20000E9471198FEB1CE00E9487198AE10E94B1
:102E3000E719A8EFB3E0E3E8F2E00E94011D0E9469
:102E40006919E6E9FFE30E9471198A98AFE7B2E0D9
:102E50009C9192FF04C0829B10C09B7F9C9382999F
:102E60000CC084E69F9399270E94711A9F918299C2
:102E700004C094609C930E9442170C94E516C0987D
:102E8000C1980895A0E6B0E00E94261C8AE08093D5
:102E9000890208950E94AA168AEF90E00E94711A92
:102EA000A0E3B0E00C9102FB0EF418C08FE711E034
:102EB0000E948719E8E9FFE30E9471198FEB11E086
:102EC0000E948719EAEAFFE30E9471190E94AA167C
:102ED00084E690E00E94711A0C9450170E947819B1
:102EE000089500918002053010F00C947F17ACE833
:102EF000B2E0E6E2FBE30E94161C0C94031800917A
:102F000080020A3010F00C948D17ACE8B2E0EEE3CA
:102F1000FBE30E94161C0C940318009180020F30F2
:102F200010F00C949B17ACE8B2E0EEE1FBE30E94DA
:102F3000161C0C94031800918002043110F00C94BC
:102F4000A917ACE8B2E0E2E4FBE30E94161C0C9483
:102F5000031800918002093110F00C94B717ACE807
:102F6000B2E0E6E4FBE30E94161C0C940318009107
:102F700080020E3110F00C94C517ACE8B2E0EAE420
:102F8000FBE30E94161C0C9403180091800203328C
:102F900010F00C94D317ACE8B2E0EEE4FBE30E942F
:102FA000161C0C94031800918002083210F00C9447
:102FB000E117ACE8B2E0E2E5FBE30E94161C0C94DA
:102FC0000318009180020D3210F00C94EF17ACE85A
:102FD000B2E0E6E5FBE30E94161C0C940318009196
:102FE0008002023310F00C94FD17ACE8B2E0EAE581
:102FF000FBE30E94161C0C940318ACE8B2E0E2E27A
:10300000FBE30E94161C08950F921F922F923F928D
:103010004F925F927F92AF92BF920F931F932F9325
:103020003F934F935F936F937F938F939F93AF9350
:10303000BF93CF93DF93EF93FF938FB78F938BB7AC
:103040008F7B8BBF80917F028F7B80937F02DB9988
:103050000C943518D39ADB9A0E94931984E690E079
:103060000E94711A8CE00E94ED198C9AE0E0F0E069
:10307000AEE6B0E00E94711DE1E0F0E0AFE6B0E046
:103080000E94711DE2E0F0E0A0E7B0E00E94711D37
:1030900002E010E0AFE6B0E04D9155270E945019D4
:1030A000AAE8B2E00D931C93AAE8B2E00D911C913E
:1030B00041E050E0041B150BA0E1B0E08D919C9124
:1030C00099BD88BD0E94A8188FE711E00E9487195A
:1030D000ECEBFFE30E9471198FEB11E00E9487195E
:1030E000EEECFFE30E9471190E94AA16E2E0F0E004
:1030F0000E948A1982990C948C188FEF93E099BDE5
:1031000088BD87E080936E008AE080936F008AE03C
:10311000809370000E94AA168F918FBFFF91EF914C
:10312000DF91CF91BF91AF919F918F917F916F91DF
:103130005F914F913F912F911F910F91BF90AF9051
:103140007F905F904F903F902F901F900F90189519
:10315000A0E7B0E00D9111274FE050E0040F151FDC
:10316000AAE8B2E00D931C93AAE8B2E00D911C917D
:103170004FE050E004231523AAE8B2E00D931C931E
:10318000AAE8B2E00D911C9140E750E0040F151F32
:10319000AAE8B2E00D931C93A0E7B0E00C911127D0
:1031A000222733274FE050E060E070E00E94E41CEB
:1031B000ACE8B2E00D931D932D933D9394E0ACE801
:1031C000B2E00E94FD1BACE8B2E00D911D912D9183
:1031D0003C9144E550E060E070E00E94E41CACE803
:1031E000B2E00D931D932D933D9389E2F6D080912B
:1031F0008A02F3D080918C02F0D088E2EED008955C
:10320000F894FFCFED91FC91EF5FFF4FFC93EE93AD
:103210000895ED91FC91E150F040FC93EE930895F8
:1032200009D00E94C11B00FC10D0089503D01ED00D
:1032300001F8F9CF0024E89457FF02C009D0689440
:1032400000F80BD010F80124089502D009D0089599
:10325000509540954F5F5F4F0895E89417FF08958C
:10326000009510950F5F1F4F68940895352F242FF8
:10327000E894452B11F468940895512F402F0027AE
:10328000112780E1440F551F001F111F021B130B54
:10329000416018F4020F131F4E7F8A9599F7089525
:1032A00014D081F0002E112E415050400ED009F460
:1032B00008954F935F93402D512D0E94C11B5F9144
:1032C0004F91F2CF01E0112708958827842B852B99
:1032D0000895A8EFB3E08D91882311F078D0FBCF4B
:1032E00008950E940E1C802D11F071D0FACF089520
:1032F00081E073D015D080E870C08FE7213039F0BD
:103300008FEB223021F08FE8233009F08FEC810F12
:103310000C94ED1988EE93E0E4D03197D9F7089535
:1033200083E09927DEC08AEF90E00E94711AD49A58
:10333000D59AD69AD79AA19AA09AA89885E090E0B3
:103340000E94711AA998DC98DD98DE9ADF9AA99AF2
:10335000EF93FF93E5E1F0E00E94651AFF91EF9192
:10336000A998BCD0A99AEF93FF93E5E1F0E00E9401
:10337000651AFF91EF91A998B1D0A99AEF93FF93A5
:10338000E5E1F0E00E94651AFF91EF91A998A6D0BF
:10339000DF98A99AEF93FF93E5E1F0E00E94651AA8
:1033A000FF91EF91A9989AD089E217D084E115D0C6
:1033B00085E513D08DE611D088E70FD088E20DD0D7
:1033C00088E20BD08EE009D086E007D00895A89A55
:1033D000829505D004D082D00895A898F9CF85951C
:1033E00010F4DF9A01C0DF98859510F4DE9A01C0D1
:1033F000DE98859510F4DD9A01C0DD98859510F46E
:10340000DC9A01C0DC98A99AEF93FF93E5E1F0E024
:103410000E94651AFF91EF91A998089500FC05D0CC
:10342000089530D005D001F8F9CF37D03FD00895B6
:10343000842F952FA62FB72FE894452B462B472B8B
:1034400011F468940895402F512F622F732F002795
:10345000112722273327F0E2440F551F661F771FDD
:10346000001F111F221F331F081B190B2A0B3B0BB8
:10347000416028F4080F191F2A1F3B1F4E7FFA9541
:1034800059F708950024E89477FF02C006D06894A5
:1034900000F809D010F80124089512D04F5F5F4F53
:1034A0006F4F7F4F0895E89437FF0895009510956A
:1034B000209530950F5F1F4F2F4F3F4F6894089511
:1034C000409550956095709508953197F1F708955E
:1034D000689462F80895E89462F8089581E090E0B5
:1034E00000C0EF93FF93EE27E82BE92B31F0EAEFD2
:1034F000F0E03197F1F70197D1F7FF91EF9108953F
:10350000A9E9B2E0E6E9F2E00E94B51A33970C941B
:10351000A31AE2EAF2E0A3E9B2E00E94911AADE058
:10352000BB27868197810E944E1C0D9383819481D5
:103530000E944E1C0D93808191810E944E1C0D9320
:103540000895EDE0FF2782810E94431C8AE38D935A
:1035500081810E94431C8AE38D9380810E94431CD9
:1035600088278C930895EDE0FF2781810E94431CFA
:103570008CE58D9380810E94431C8CE58D93828124
:103580000E94431C88278D93089593E0ADE002C00C
:1035900096E0AAE0B0E08FB7F89401910D939A9568
:1035A000E1F78FBF08950191119145EB55E00E941D
:1035B0001619440F440FF42E0F31150728F481E03B
:1035C000E82E0395D02E22C00C33150728F482E094
:1035D000E82E0E51D02E1AC00150150B4DE651E0C9
:1035E0000E943619F40E7CE07A95872F9927EEE039
:1035F000F6E3A2E1BB270E941E1C02171307A0F3EB
:103600007395E72E021B130B0395D02E089500002F
:103610001F003B005A0078009700B500D400F3006B
:10362000110130014E01019111912191308140E849
:1036300051E561E070E00E94111A042F152F0C94DF
:10364000D51AA3DF0E2D0A95802F0295003220F0A7
:103650001F2D137009F40395DA940D0D1127992786
:10366000E2E7F6E3A8E1BB270E94231C080F111F25
:103670000895000F1B2A384755647381909E0E945D
:10368000131B0C94221B81DF0F2D11274CE35527B0
:103690000E94101955270E0D151F4CE322273327C2
:1036A000662777270E94CB1B0D0D131F231F08953C
:1036B0006CDFDF92EF92FF920F2D11272227332725
:1036C0004DE651E060E070E00E94CB1BFF904F2D73
:1036D0004D5F469546955527662777270E94E41C3F
:1036E000EF90DF900F931F932F933F930E94221B25
:1036F000222733277F916F915F914F910C94E41CA7
:1037000047DFAF92BF92CF920E94591B40E851E52C
:1037100061E070E00E94CB1BFF90EF90DF900F9371
:103720001F932F933F930E94441B7F916F915F9152
:103730004F910C94E41C019111912191308140E84A
:1037400051E561E070E00E94111A0C94AB1B0191ED
:1037500011912191308140E15EE060E070E00E94D3
:10376000111AF42E4CE350E00E941619E42ED02ECC
:103770000895AF93BF930E949B1BBF91AF910C9490
:10378000A11A0F92B801469F8001479F100D569FC6
:10379000100D0F9008950F921F922F92C801D9011A
:1037A000489F80014A9F90014B9F202C499F100DFC
:1037B000211D321D5A9F202C589F100D211D321D96
:1037C000599F200D311D689F200D311D699F300DBF
:1037D000789F300D2F901F900F9008950E940E1C1F
:1037E0000D920020D9F70895369A3699FECF369A71
:1037F0003699FECF84B195B10895903071F00D9156
:103800001D912D913C9136952795179507959A9581
:10381000D1F73C932E931E930E930895C89531963D
:103820000020089591E005C092E003C094E001C03B
:1038300098E0F4DF0D929A95E1F70895880F991FAB
:10384000E80FF91FF1CFE80FF91FECCF82E001C0BC
:1038500084E099279D938A95E9F7089591E088235C
:1038600021F08894991F8A95E9F7892F90950895FA
:10387000BB270E942E1C9C9198279C933197F1F7AF
:1038800098279C93089500278A3018F08A50039552
:10389000FBCF005D0D93805D8D9308958053905311
:1038A0000027813018F0065F8A95FBCF090F089535
:1038B000AF93BF930F939F938F938FB78F93A3E98A
:1038C000B2E08C9183958D938C3309F03DC08827AD
:1038D0008E9311968C9183958D938C3309F034C01F
:1038E00088278E9311968C9183958D93883161F5FD
:1038F00088278E9311968C9183958D939C910EE1E0
:10390000943089F0963079F0993069F09B3059F015
:103910000CE1923039F411969C911197937019F43F
:10392000039501C00FE1801778F071F081E08E936C
:1039300011968C9183958D938D3031F481E08E9327
:1039400011968C9183958C938F918FBF8F919F91BE
:103950000F91BF91AF910F921F922F923F924F9272
:103960005F927F92AF92BF920F931F932F933F93DB
:103970004F935F936F937F938F939F93AF93BF9377
:10398000CF93DF93EF93FF938FB78F930E94AE1582
:103990008F918FBFFF91EF91DF91CF91BF91AF9149
:1039A0009F918F917F916F915F914F913F912F9157
:1039B0001F910F91BF90AF907F905F904F903F907D
:1039C0002F901F900F901895040F151F261F371F5B
:1039D0000895041B150B260B370B089504171507C4
:1039E000260737070895000F111F221F331F089560
:1039F00000951095209530950F5F1F4F2F4F3F4F2B
:103A00000895019110810EC0019111912191308191
:103A10000BC00191108117FF05C03FEF2FEF04C0CD
:103A2000008111272227332737FF03C0E1DF8DE212
:103A30008D93CF93DF93CF92DF92EF92AA24BB2492
:103A4000CC24DD24EE2440E2CAE0DD2755E093E3F8
:103A50008881890F87FD9F7083FD907F891B8993E3
:103A60005A95A9F7C0DFAA1CBB1CCC1CDD1CEE1CA0
:103A70004A9551F7E894EFE0FF2782910ED0EB30A2
:103A8000E0F71EF068948A2D0CD088278D93EF9074
:103A9000DF90CF90DF91CF910895982F829501D03C
:103AA000892F8F70805D26F0803309F40895689423
:103AB0008D930895E199FECFEEBBFFBB319608953B
:103AC00091E001C092E07B3751F47FB7F894F2DFC8
:103AD0008D918DBBE29AE19A9A95C9F77FBF7727BE
:103AE000089591E001C092E0E5DFE09A8DB38D93F7
:103AF0009A95D1F70895FF93881BF9E0001FFA9576
:103B000011F4FF910895881F841B18F4840F889482
:103B1000F5CF0894F3CFFFFFFFFF0F0000000A006E
:103B200000008051010001000000630000001D0042
:103B300000000F2700007F33E1017F5101000500E5
:103B400000001E0000003C0000002C010000580294
:103B50000000100E000050460000A08C00005761CD
:103B6000727465206269732053746172742000005E
:103B70005370696567656C766F726175736C2E2022
:103B8000000042656C69636874756E67000050617F
:103B90007573652020202020000042696C646572E6
:103BA0002020202000002042617474657269652025
:103BB0006C6565722021000020426974746520776D
:103BC00065636873656C6E20000042617474657291
:103BD0006965207363687761636800002020426133
:103BE000747465726965204F4B20202000002020EE
:103BF0007374617274652054696D657220200000D1
:103C0000202054696D657220626572656974202098
:103C100000004D656E7565206175737784686C650D
:103C20006E2000002053656B756E64656E20000089
:103C30002020202020202020202020202020202084
:103C4000000050726F6700002042656C6963687401
:103C5000756E67002050617573652020202020005C
:103C60006175746F6D2E204175736C9473656E2051
:103C7000000050726F6772616D6D206265656E64E1
:103C800065740000205374616E646279204D6F6426
:103C90007573202000002057617274652000204A4F
:103CA00065747A7420002020535641202000205350
:103CB000686F6F7420007A656974672E2041757390
:103CC0006C9473656E20000057657274652067659B
:103CD0007369636865727420000050726F67722E9A
:103CE0002067656C94736368742000005A6569747A
:103CF000702E2067656C94736368742000002056F2
:103D0000657273696F6E2020312E312E34200000D1
:103D100030322E30382E3230303920233346453081
:103D2000000044616E6B20616E204C756369616EAA
:103D30006F2C00005069742026204D53636877650E
:103D4000697A657200002020466F6B757373696530
:103D500072656E20202000002020202020456E74F7
:103D600065722020202020200000204175736C9473
:103D700073656E2053746172742000002042656C7C
:103D80006963687465002053746F70206D697420D6
:103D9000456E7465722000007300206D69742046C2
:103DA0006573747374656C6C20200000206D616E07
:103DB0002E204175736C9473656E20200000456E53
:103DC00074657220756E642068616C74656E0000A5
:103DD000204175666E61686D65206C84756674201F
:103DE00000002042656C6963687465200000206FE4
:103DF000686E6520466573747374656C6C20000092
:103E00004D656E7565206F64657220456E746572D0
:103E100000002045696E7374656C6C756E67656E25
:103E2000202000002050726F6772616D6D7A6569A5
:103E300074656E2000002020205A65697470756ECC
:103E40006B7465202020000020202046756E6B7466
:103E5000696F6E656E202020000020204C434420B6
:103E60004B6F6E747261737420200000204C4344C9
:103E70002048656C6C69676B6569742000006D6132
:103E8000782E2048656C6C69676B6569742000004A
:103E90002020556872207374656C6C656E2020203C
:103EA0000000202053564120616B746976203F202A
:103EB000202000002020202020206E65696E202018
:103EC000202020200000202020202020206A6120A7
:103ED000202020202020000020506F776572205481
:103EE000696D656F757420200000204D696E7574D2
:103EF000656E00002053656B756E64656E00206909
:103F00006E732048617570746D656E756520000074
:103F1000204175736C9473657A6569742000202064
:103F2000202020204E2F4120202020202020000073
:103F3000202B00002020417573736368616C7465E9
:103F40006E202020000050726F67722E206C9473D8
:103F50006368656E203F00005A656974702E206C9E
:103F600094736368656E203F000057657274652026
:103F700073706569636865726E2000002020496E69
:103F8000666F726D6174696F6E202020000073206F
:103F900000006E200000200020204269747465201B
:103FA0005461737465202020000020206C6F736CB6
:103FB000617373656E20212020200000556E6976A4
:103FC000657273616C2054696D65722000006279BE
:103FD000205069742026205454203230303700009D
:00000001FF
